:020000001728BF
:08000800172863308C000C2066
:100010008D0B052800000800000000000000000013
:100020000000000000008C0B0C2800000800831664
:100030000030810000308B00831600308500433093
:10004000860081178312030185008600FF308E0031
:10005000FC308F008E030514851005114620051411
:1000600085140511462005108514051146208F0BB7
:100070003A284928051085140515462005108510D5
:100080000515462005148510051546200E088D001F
:10009000052005148510051103308D00052005107D
:1000A0008514051103308D000520051085100515F8
:1000B00003308D000520492805118510061C612894
:1000C0005E288515FA308D0005208511FA308D00E7
:0400D00005205E2881
:00000001FF
